:020000040000FA
:040000008B17FD2934
:08000800FB000308FC000A08DC
:10001000FD008A1183120B1D1628FF0803191228F0
:10002000FF0315287E148B12FF250B117D088A0013
:100030007C088300FB0E7B0E09000008A00008006E
:10004000840A00088403A1001D28840A840A000889
:1000500084038403A20020282008800008002108CF
:10006000840A800084032C282208840A840A8000E1
:10007000840384032F280008A0070800840A0008CE
:100080008403A107031C3B28A00A3B28840A840A96
:10009000000884038403A207031C3E28A10A031D51
:1000A0003E28A00A3E280008A0020800840A000892
:1000B0008403A10203185328A0035328840A840A46
:1000C000000884038403A20203185628A103210A0E
:1000D000031D5628A00356280008200208006C20A3
:1000E000031D0800840A00082102080000082006F9
:1000F000803903196C280314A01B03100800762014
:10010000031D08007228A01BAE280800A01BC328EE
:100110000800A30A031D0800A20A031D0800A10A83
:10012000031D0800A00A0800A01BB528A028A01BDA
:10013000B528A228A01BB528A528A01BB528A9284A
:10014000A0099228A009A1098F28A009A109A20944
:100150008C28A009A109A209A30989287F30A00041
:10016000FF30A100FF30A20008008030A000003066
:10017000A1000030A2000800FF30A000FF30A10065
:10018000FF30A20008000030A0000030A1000030C5
:10019000A2000800A01B8038E028A101A201A30151
:1001A000A4000310A30DA20DA10DA00D0318DB28C0
:1001B000A01BAE28DD28A01FB528A40BD12808005D
:1001C000A5007F39A400250DA00CA10CA20CA30C46
:1001D000A40BE3280800A101A201A301A4000310BD
:1001E000A30DA20DA10DA00D0318BC28A40BEF2890
:1001F0000800A01B0729A008031DAE282108A000A5
:100200002208A1002308A200A01BAE280800200A93
:10021000031DB5282108A0002208A1002308A20080
:10022000A01FB5280800A008031DBC282108A000B5
:100230002208A1002308A20008002208A300210828
:10024000A2002008A100A001A11BA0030800220811
:10025000A3002108A2002008A100A0010800A0011D
:10026000A10100380319080003100018A007A00C12
:10027000A10C8018A007A00CA10C0019A007A00CCD
:10028000A10C8019A007A00CA10C001AA007A00CBB
:10029000A10C801AA007A00CA10C001BA007A00CA9
:1002A000A10C801BA007A00CA10C0800801F2F2907
:1002B0008009800A2F218009800A9728A400840AD7
:1002C0002F212108A3002008A2008403240856211E
:1002D0002208A1070318A00A2308A200080020088A
:1002E000A200210856212108A6002008A500220806
:1002F0005E21A401A51BA403243084004628A40089
:10030000840A2F212108A3002008A20084032408C6
:100310002F212208A1070318A00A2308A200080021
:100320002008A20021082F212108A6002008A500EE
:1003300022087F21A401A51BA403243084004628A1
:100340000008A200840A0008A3002208230403195D
:10035000B329A21BB329A01BB3290310A30DA20D1F
:10036000A10DA00DA9292208B529A200A3012430BE
:1003700084002C20A5010830A000263084002C2009
:10038000A001A1010310A20CA30C223084003E2086
:100390002008240203190310A50D2518D2292230A4
:1003A00084005620A60BC2292508A00008002108B9
:1003B000A3002008A2003E20801BE42922308400F4
:1003C0006F20031CBC280800223084006F20031813
:1003D000C32808002108A3002008A2003E20801B9B
:1003E000F729223084007F20031CAE280800223029
:1003F00084007F200318B528080083120730990075
:100400008312831600309F008312831671308F0091
:1004100083128130840080128011813084000014A6
:1004200080140015001000112A2A2008FF00210462
:100430000319A10A2108003C81000318FF030B11D6
:100440008B167E100800FF0081011F2AFF01003C6F
:1004500081001F2A83129010101690163D2A8E01DB
:100460008F0110140C1008000F08A0000E08A10046
:100470000F082002031D342A0800831283128C13F4
:100480005E2A83169B005C2A83161C1483161A08A6
:100490005C2A83161B085C2A83169B0A5C2A831637
:1004A0009B035C2A83169B075C2A44228000840AF3
:1004B0004C22A003031D552A831208008312652ACB
:1004C000FF30A000FF30A100080083161F169F1602
:1004D0001F178E2AA0002030840083129F011F1452
:1004E0000018782A83161F14812283161F107E2A73
:1004F0001F1583169F14812283169F108312A0005C
:1005000008000A30FF3E031D822A83129F149F18A1
:10051000872A83121E0883121F1008008312C02A24
:10052000A2002230840020082F212108A2002008E8
:1005300052224422A3004C224422A4002408A100F9
:100540002308A0002208A2002108A4002008A3007C
:10055000FF30A00022308400532023308400200884
:100560002F212108A6002008A500223084001D208C
:100570002430840020082F21253084003E200800EC
:10058000831605118512950183128312D125202629
:1005900043260030A000200841220830A0002C3063
:1005A00084005522B40185122F2264226022FF307C
:1005B000A400243084006C20031DC92A0F08A00069
:1005C0000130EB202E3084006C200318D22A222622
:1005D000031CD62A3608A9003508A80034222F2289
:1005E000353084002F20B40A343084001D200330BD
:1005F000A400243084006C200318FF2AD62A35304A
:1006000084002020283084003E20353084002F20B4
:100610008326D1259326B401BB01BC012F08BD0060
:10062000FF30A000FF30A100373084002F2064226B
:10063000E030A000200864221030A0002D1CA00A89
:10064000200864224426031D2E2B4426031D2E2B36
:100650000D30A000200841224422A000200864227E
:100660004E3084002C20283084002C203030A00014
:100670004F3084002C200C30A0002830840020084B
:100680002F2113214F3084003B204F3084002C2039
:10069000200841224422A0003E3084002C204C221D
:1006A0000B30A0005030840055220830A0005208C2
:1006B000B5215C3084002C200830A0005108B52101
:1006C000513084002C2065237B2BD701A0016B23A4
:1006D000571F672B080057081F39A03E84002008C9
:1006E0008000D70A0800200957071F39A03E840060
:1006F0000008A00008000F08A0003D3084006C2016
:1007000003188C2D2226031C7B2BB41F8D2B342227
:100710002F22393084003E20AE2B34222F22393054
:1007200084002F20353084005620A01BA2202830C2
:1007300084002F203930840020200130EC20353017
:1007400084005620A01BA220283084006F2039305E
:10075000840020200318AE2BB4177B2B3530840087
:100760002F200330EC202C18B72B20086422B41360
:10077000353084001D202B213B3084003E203B304F
:1007800084002F20341B232CE425832662252C187B
:10079000CB2B200864223F08C900E1234A308400A3
:1007A0001D20323084006C20031CD92B3230840091
:1007B0001D204A3084002C202C18E02B20086422B5
:1007C0007B2B3B30840020200130A400F430A500B6
:1007D000243084006F2003180B2C35308400202037
:1007E000373084006F200318002C373084002F200E
:1007F000B401503084001D204A3084002C200800B1
:10080000B40A343084001D200530A4002430840054
:100810006C20031CF92BB4013417B701B80149301F
:1008200084001D20553084006C20031C182CB0015E
:10083000DD01DE01DF01DA01DB01FF30A00058300D
:1008400084002C2008008516B41E2A2C4B1D342C45
:100850001926342CE425353084001D2030308400E6
:100860006C20031C342CB416333084001D2035302A
:10087000840020087F210330A4000030A50024302C
:1008800084006F20031C482C0330A0000030A1001E
:10089000283084002F203530840020202830840028
:1008A0005620393084002F20373084002020353006
:1008B00084003E20373084002F20A82662252C1883
:1008C000632C200864223530840020200330EC2083
:1008D000563084002C204130840020200330CE206C
:1008E0006B23A801A9010030A0002A3084002C202D
:1008F00073232121283084003E20283084002F20BB
:100900002A3084001D20A00A0530A4002430840071
:100910006C20031C752C2830840020200530CE204C
:100920005E3084002C202830840020205A3084003F
:100930005620F920603084002C20A01BA0205D30C0
:1009400084002C202908DB002808DA000830A000E9
:100950004F3084003B20200841227F30A0005E30D1
:1009600084005320523084006C20031CBA2C523077
:1009700084001D205E3084003B2086205C30840093
:1009800020082F210530EC20283084002C205D30F9
:1009900084001D205130840020082F210530EC20D8
:1009A000033090222830840020082F210630E020D8
:1009B0009720283084002F205830840020202830B1
:1009C0008400D721583084002F2050308400200824
:1009D0002F210A30A400243084006C200318F22C4C
:1009E0000A30A0004A3084002C205D3084001D2095
:1009F000533084006C20031C0B2D4A3084001D20D2
:100A0000543084006C20031C082D543084001D20B9
:100A10004A3084002C20373084001D202F30840081
:100A20006C20031C1B2D2F30840053203730840092
:100A30002F20F030B4053B30840020200330A40088
:100A4000E830A500243084006F200318372D49308A
:100A500084001D203F3084005320A01BA0200930BB
:100A6000A400243084006C20031834163E2D341A60
:100A70003E2D4E3084001D2056253E2DB41AD4251F
:100A8000FF30A000CB1B472D4A3084001D202C18BE
:100A90004B2D200864223422393084006F20031C3F
:100AA0004B2D85122C1D7B2B16267B2B20084122DB
:100AB0002830A000200852224422A0004A3084009E
:100AC0002C2008002D3084001D200430A400243088
:100AD00084006C200318862D20088A0005308A06C1
:100AE0000A068A06763E03188A0A82007A2D7E2D2F
:100AF000842D852D3F3084001D2008004130840066
:100B000020200330CE200800080008002008593EAD
:100B100084000008A0000800851613264130A000BC
:100B20008F3084002C20B501B6014A3084001D208E
:100B3000AC1C9C2DE530A0000330E0204A3084003E
:100B40002C200515353084002020A10A031DA92D75
:100B5000A00A353084002F200330A4002430840004
:100B60006C20AC1CB82D0A30A400243084006C200A
:100B700003180028013084001D201F30A0054A30D2
:100B800084006C20031CBA2D0511013084001D2047
:100B90001F30A0054A3084006C200318C52D0515B0
:100BA000A22DCA01CC01132EF5254C3084002C2037
:100BB0004B180800CC080319080005154B14CB147A
:100BC0000830E02015220800F52535308400200883
:100BD0007F2115220515CB010800A0080319080084
:100BE00015220515CB14CB1708001830A0002008DB
:100BF00041224A3084001D200F30902208004B1CF7
:100C0000132ECB180C2ECB144B19072E05154C08A0
:100C1000FF3C81008B160800CB10CB1305114C084C
:100C200081008B160800CB01051108004B1505113A
:100C300008004B1D08004B11CB1C080005150800CF
:100C4000851608000314051A0310CD0C03182E2E68
:100C50004D10E0304D0203184D1408004D141030B3
:100C60004D02031C4D10031008000314051A031055
:100C7000A001A00D200864220B30A00020086422EF
:100C8000200864220800080000306A222B21283046
:100C900084002F200C30A000200841224422A00014
:100CA0002A3084002C200E30A00020084122AB0105
:100CB0004422A000FF30A400243084006C200319DB
:100CC000742E2B21283084005620F920A01BA02050
:100CD0002A3084006C20031C702EAB0A4C22582E44
:100CE0002B08A000031108000800442620086422F5
:100CF000283084001D2020086422293084001D2013
:100D0000200864220800BF01C001C101C101C20165
:100D1000C301C830A0002B2135308400A0213F3012
:100D200084002C200800313084001D200130EB208D
:100D3000473084002C20313084001D203130840065
:100D400020082F210430EC20483084002C2008009B
:100D50000630A0004730A100AE30A2002830840049
:100D600034203530840020203F30840090218320BF
:100D70000530CA20F920A520283084004620F9201B
:100D8000453084002F20473084001D2045308400EA
:100D900020085E210530CA203F3084003E203F30CD
:100DA00084002F20353084002020413084006F21C2
:100DB0000730CA20F9203F3084003E203F308400B5
:100DC0002F203E3084001D204A30840020082F212F
:100DD0002B21CB1FFC2E4630A0003E308400200883
:100DE0002F212B21283084002F203E3084001D200D
:100DF0002B21283084003E208320A2203F30840015
:100E00003E203F3084002F20483084001D20453094
:100E1000840020085E210330CA20433084002F2044
:0E0E2000413084003E20413084002F20080025
:02400E00D430AC
:10420000000001000E001100FF002300C800820022
:084218000500010048006D00E3
:0242200092000A
:1042300014001E002D003C0044005500660077006D
:1042400088009900AA00BB00CC00DD00EE00FF0052
:0E42500005002D0055007D00A500CD00F500F5
:1042600078005000320032001400320000000000DC
:1042700000003200500064006E007800320032000E
:104280001400320000000000000032005000640002
:104290006400A00032003200140032000000000070
:0842A000000032005000640030
:00000001FF
